:100000000C940B010C9475110C944E110C94271147
:100010000C9400110C9433010C9433010C94D910FE
:100020000C9433010C9475120C9474140C94E61413
:100030000C9433010C9433010C9433010C94330170
:100040000C9433010C9433010C9433010C94330160
:100050000C9433010C9433010C9433010C948F10E5
:100060000C9433010C94B80E0C94920E0C94330142
:100070000C9433010C9433010C9433010C94330130
:100080000C9433010C9433010C9433010C94330120
:100090000C94600A0C9433010C9433010C943301DA
:1000A0000C9433010C9464080C943301200E230E3D
:1000B000120E160E1C0E440E440E440E270E2B0E6E
:1000C0002F0E350E390E440E3F0E41627374616E71
:1000D000643A20256420256420256420256420209E
:1000E000204C696E69653A202564202564202564CA
:1000F0002020205765673A20256420256420202091
:1001000057696E6B656C3A2025642020205A65691A
:10011000743A2025640000000000240027002A0013
:100120002D00300000000000250028002B002E00CC
:100130003100000000002300260029002C002F00C1
:10014000040404040403040502020202040302027C
:10015000020206060606060604040202020404045D
:1001600008020110408040102040804080080204B6
:10017000018040201002011080102040402000002B
:10018000000200090F0000030401000C0000000041
:1001900000000000000000000000000000080B004C
:1001A000020202010009040000010202000005240D
:1001B00000100105240101010424020605240600A3
:1001C000010705810310004009040100020A000034
:1001D00000070502024000000705830240000004FA
:1001E00003090412010002EF02014041233680009E
:1001F000010102030141726475696E6F204C4C432A
:100200000041726475696E6F204C656F6E61726437
:100210006F00A720482111241FBECFEFDAE0DEBF18
:10022000CDBF12E0A0E0B1E0E8E7F1E502C0059043
:100230000D92AE39B107D9F725E0AEE9B2E001C0C1
:100240001D92AC3EB207E1F711E0CAE0D1E004C074
:100250002197FE010E949C25C930D107C9F70E9451
:1002600051170C94AF280C940000809100058F3F2B
:1002700061F061E00E94430F60E0809100050E9400
:10028000130F8BE193E00197F1F708954091070573
:10029000209105053091060590E0941749F02D5FF7
:1002A0003F4FF90133975081581721F09F5FF5CFE9
:1002B0008FEF0895892F089584E00E944601909160
:1002C0000705891758F4E0910505F091060593E0BC
:1002D000899FE00DF11D11248281089580E0089529
:1002E000CF93DF93009779F0FC0101900020E9F7AC
:1002F0003197AF01481B590BBC0183E094E00E9489
:10030000020DEC0102C0C0E0D0E042E050E067E442
:1003100072E083E094E00E94020D8C0F9D1FDF913C
:10032000CF910895FF920F931F93CF93DF93CDB793
:10033000DEB7A0970FB6F894DEBF0FBECDBF8C011D
:10034000F62E8FEF860F823088F4809100058F3F64
:1003500079F061E00E94430F61E0809100050E9406
:10036000130F8BE193E00197F1F702C00E94350172
:10037000E091F304F091F4040190F081E02DB801D4
:1003800083EF94E009950E94350162E0F61231C0D6
:10039000E091F304F091F4040190F081E02DBE01AE
:1003A0006F5F7F4F83EF94E0099540E08091FF04F9
:1003B0004817F8F4242F30E0220F331FF801E20F22
:1003C000F31FA1E0B0E0AC0FBD1FA20FB31F8091DF
:1003D0000105909102052D913C91BC01621B730BAC
:1003E0009B0180819181280F391F318320834F5FCA
:1003F000DDCFA0960FB6F894DEBF0FBECDBFDF9164
:10040000CF911F910F91FF90089591E09093020476
:1004100080931205109201041092000408959091A7
:10042000DD039111FCCF613208F060E291E090931E
:10043000DD039093DC032FEF2093DB031092DA03AC
:10044000260F2093D9039093D8039091D803880F57
:10045000892B8093D8038091D703813061F4109267
:10046000D7038091D8038093BB008091BC0083FDAB
:10047000F8CF85EC01C085EE8093BC008091DD0350
:100480008130E1F38091DA03861710F46091DA038A
:10049000A7EBB3E020EE33E0F9018E2F821B861725
:1004A00018F48D918193F9CF1092DF036093DE03EE
:1004B000862F08952091000490911205213208F0B2
:1004C0004AC08091DD038111FCCF32E03093DD031F
:1004D00031E03093DC033FEF3093DB031092DA031B
:1004E0002093D903A7E9B3E047EB53E0FA013E2F8D
:1004F000341B321718F43D913193F9CF1092D80381
:100500002091D803990F922B9093D8039091D70301
:10051000913061F41092D7039091D8039093BB006F
:100520009091BC0093FDF8CF95EC01C095EE9093AF
:10053000BC009091DD039230E1F39091DB039F3F8B
:1005400079F08091DB03803241F08091DB038033CE
:1005500031F084E005C081E003C082E001C083E0A7
:100560001092010410920004109202040895BF92A8
:10057000CF92DF92EF92FF920F931F93CF93DF936F
:100580008091B5040E94050268EA80EA94E00E9426
:100590000E080E945A0266E08091B5040E940F0284
:1005A0000E9483107B018091DE0390E02091DF03A5
:1005B000821B91090697ACF48091B6049091B70420
:1005C000892B89F30E9483106E197F098091B604EC
:1005D0009091B7048617970730F781E08093B804AD
:1005E00033C080EA94E00E94C207C82E80EA94E0FB
:1005F0000E94C207B82E80EA94E00E94C207E82E4B
:1006000080EA94E00E94C207D82E80EA94E00E941B
:10061000C207F82E80EA94E00E94C2071B2D00E07A
:100620000C291093AD040093AC04DD2D20E0C22F03
:10063000CE29D093AF04C093AE04982F88278F297A
:100640009093B1048093B004DF91CF911F910F91EB
:10065000FF90EF90DF90CF90BF9008950F931F937E
:10066000CF93DF93082F162FCCEAD4E089850E9420
:100670000502602F80EA94E00E940E08612F80EA54
:1006800094E00E940E080E945A028E83DF91CF915F
:100690001F910F910895CF93C82F0E9405026FE01C
:1006A00080EA94E00E940E080E945A0281110FC055
:1006B00061E08C2F0E940F029091DE038091DF0396
:1006C000981729F080EA94E0CF910C94C2078FEF3D
:1006D0009FEFCF910895EF92FF920F931F93CF93C7
:1006E000DF938091D5040E9405028091D2049091FD
:1006F000D304039731F46091DA047091DB046068ED
:1007000004C06091D8047091D90480EA94E00E94FA
:100710000E080E945A028093D10466E08091D504AD
:100720000E940F020E948310EB018091DE0390E093
:100730002091DF03821B91090697ACF48091E404B9
:100740009091E504892B89F30E9483106C1B7D0B2B
:100750008091E4049091E5048617970730F781E0D3
:100760008093E60474C08091D2049091D3040397DF
:10077000F9F480EA94E00E94C207182F80EA94E01E
:100780000E94C207E82E80EA94E00E94C207D82F98
:1007900080EA94E00E94C207F82E80EA94E00E946A
:1007A000C207C82F80EA94E00E94C207082F39C010
:1007B00080EA94E00E94C207E82E80EA94E00E945A
:1007C000C207182F8091D2049091D304892BA9F4E9
:1007D00080EA94E00E94C207F82E80EA94E00E942A
:1007E000C207D82F80EA94E00E94C207082F80EA4F
:1007F00094E00E94C207C82F14C080EA94E00E94CF
:10080000C207082F80EA94E00E94C207C82F80EA3E
:1008100094E00E94C207F82E80EA94E00E94C2078A
:10082000D82F212F30E03E293093C0042093BF04FD
:100830002D2F30E03F293093C2042093C1042C2F88
:1008400030E0C901902B9093C4048093C304DF91DE
:10085000CF911F910F91FF90EF900895BF92CF928B
:10086000DF92EF92FF920F931F93CF93DF938091CC
:10087000D4040E94050268EA80EA94E00E940E080F
:100880000E945A028093D10466E08091D4040E94B1
:100890000F020E9483107B018091DE0390E0209183
:1008A000DF03821B91090697ACF48091E4049091D8
:1008B000E504892B89F30E9483106E197F098091CA
:1008C000E4049091E5048617970730F781E0809360
:1008D000E60433C080EA94E00E94C207C82E80EA92
:1008E00094E00E94C207B82E80EA94E00E94C207FA
:1008F000E82E80EA94E00E94C207D82E80EA94E0B5
:100900000E94C207F82E80EA94E00E94C2071B2DC5
:1009100000E00C291093BA040093B904DD2D20E007
:10092000C22FCE29D093BC04C093BB04982F882734
:100930008F299093BE048093BD04DF91CF911F91C6
:100940000F91FF90EF90DF90CF90BF9008950F939D
:100950001F93CF93DF93082F162FC9EBD4E08C8D14
:100960000E940502602F80EA94E00E940E08612F29
:1009700080EA94E00E940E080E945A02888FDF915C
:10098000CF911F910F9108950F931F93CF93DF93F2
:10099000082F162FC9EBD4E08B8D0E940502602F23
:1009A00080EA94E00E940E08612F80EA94E00E94A1
:1009B0000E080E945A02888FDF91CF911F910F91EC
:1009C00008952091D2043091D3042330310511F0E1
:1009D000803210F40C94A7040C94C4041F93CF939A
:1009E000DF931F92CDB7DEB7182F69830E940502EF
:1009F000698180EA94E00E940E080E945A028111E7
:100A000012C061E0812F0E940F029091DE0380915D
:100A1000DF03981741F080EA94E00F90DF91CF91C7
:100A20001F910C94C2078FEF9FEF0F90DF91CF9132
:100A30001F910895CF92DF92EF92FF920F931F9331
:100A4000CF93DF93CDB7DEB72C970FB6F894DEBF08
:100A50000FBECDBF10E080910705181788F4E09114
:100A60000505F091060583E0189FE00DF11D1124A6
:100A700080818F3118F462E00E94430F1F5FEBCF3B
:100A8000809108058F3170F460E00E94130F61E0DF
:100A9000809108050E94430F8091100590911105E7
:100AA0000E947F0F8091090590910A05892B01F51D
:100AB0008CE0E8E3F1E0DE01119601900D928A9559
:100AC000E1F76CE070E080E090E00E94D7270097AB
:100AD00079F02CE0FE013196DC0101900D922A950F
:100AE000E1F790930A058093090586E080930B0552
:100AF000209105053091060580E090910705891742
:100B000050F4F90193E0899FE00DF11D1124128248
:100B100011828F5FF2CF10E080910B05181708F05B
:100B20007EC09091090580910A05E92FF82FE10F09
:100B3000F11DE10FF11DC080D18040910C05509155
:100B40000D05B60180E090E00E94031280910E0531
:100B500090910F050E947F0F00E080910705081714
:100B6000E0F483E0089F70011124E0910505F09105
:100B70000605EE0DFF1D80818F3168F40E94EA0E9C
:100B8000892B49F4E0910505F0910605EE0DFF1D56
:100B900081818F5F81830F5FE0CF0E94E911809197
:100BA0001005909111050E947F0F40910C05509106
:100BB0000D05B60181E090E00E94031280910E05C0
:100BC00090910F050E947F0F00E0809107050817A4
:100BD000E0F493E0099F70011124E0910505F09184
:100BE0000605EE0DFF1D80818F3168F40E94EA0E2C
:100BF000892B49F4E0910505F0910605EE0DFF1DE6
:100C000082818F5F82830F5FE0CF0E94E911809124
:100C10001005909111050E947F0F1F5F7DCF2C96CC
:100C20000FB6F894DEBF0FBECDBFDF91CF911F91FD
:100C30000F91FF90EF90DF90CF9008958091BB05CA
:100C4000E091BC05F091BD05882311F0849101C0AD
:100C500080819FEB980F9A3110F4805E0895803266
:100C600069F42091BC053091BD05A9014F5F5F4F2C
:100C70005093BD054093BC05232B01F708951F93A6
:100C8000CF93DF930E941E06C0E0D0E01AE090ED03
:100C9000980F9A30B8F41C9F90011D9F300D1124BD
:100CA000E901C80FD11D87FDDA95E0978091BC0559
:100CB0009091BD0501969093BD058093BC050E945F
:100CC0001E06E5CFCE01DF91CF911F9108952F929F
:100CD0003F924F925F926F927F928F929F92AF92CC
:100CE000BF92CF92DF92EF92FF920F931F93CF9319
:100CF000DF93CDB7DEB727970FB6F894DEBF0FBEF0
:100D0000CDBF9F838E831B014D838091B8058111D8
:100D10001BC081E08093B805109272001092C00051
:100D200094E09093C10099E09093C2008093C30037
:100D300083E08093BF0088EE8093D1001092BF00C3
:100D40001092D200579A789410920B012E813F8115
:100D500037FF05C03F773F832E830AE001C001E0E3
:100D600088E2089F802D112490E04E815F81481712
:100D7000590708F4C2C0013039F44131574220F01C
:100D8000E0E1F7E2FF83EE83802E912CA12CB12CC1
:100D90008E819F81969587959C0140E050E0298344
:100DA0003A834B835C834E815F812A01612C712CD5
:100DB000A501940160E072E18AE790E00E94582565
:100DC00029813A814B815C81620F731F841F951FBB
:100DD000A30192010E94BE2469017A01EE24FF243E
:100DE00010E01F5FC11434E0D306E104F10408F100
:100DF00020E032E14AE750E0012E04C055954795C6
:100E0000379527950A94D2F7C501B4010E94582559
:100E100029813A814B815C81620F731F841F951F6A
:100E2000A30192010E94BE2469017A01EE24FF24ED
:100E3000D8CF0A3049F48E819F8105966AE070E030
:100E40000E9474257F836E834E815F81483E83E0DC
:100E5000580759F09101DA010E94492528EE33E044
:100E600040E050E00E94BE2419011092720080916F
:100E7000C100807F182B1093C100BB27AF2D9E2D82
:100E80008D2D8093BF00C092D1002D81203108F0BC
:100E90002FE080E190E0821B910904C0F694E79472
:100EA000D794C7948A95D2F78D2D99278093BF0048
:100EB000C092D2003092BA052092B90589B38FEF63
:100EC00089BB84E08093720027960FB6F894DEBF4A
:100ED0000FBECDBFDF91CF911F910F91FF90EF908B
:100EE000DF90CF90BF90AF909F908F907F906F904A
:100EF0005F904F903F902F9008959F838E8344CFB3
:100F000085ED8093BC008091BC0084FDFCCF1092E5
:100F1000DD03089540919005262F30E0240F311D08
:100F200021323105DCF42091DD032430C9F4FC01C9
:100F300080E090E0861758F4309190052191DC0113
:100F4000A259BA4FA30FB11D2C930196F3CF8091F4
:100F50009005680F6093900580E0089581E0089502
:100F600082E008950895E091DF038091DE03E817A1
:100F700030F4F0E0E052FC4F808190E008958FEF74
:100F80009FEF08959091DF038091DE03981750F44E
:100F9000E92FF0E0E052FC4F208130E09F5F90931A
:100FA000DF0302C02FEF3FEFC90108958091DE03F8
:100FB00090E02091DF03821B91090895CF92DF9288
:100FC000EF92FF920F931F93CF93DF937C01262F15
:100FD000972F8A0180910204882391F0C62FD72F82
:100FE0006E01C40ED51ECC15DD0571F06991D701D7
:100FF000ED91FC910190F081E02DC7010995F3CFAF
:10100000642F822F0E948A07C801DF91CF911F9120
:101010000F91FF90EF90DF90CF900895CF93DF93E3
:101020001F92CDB7DEB76983209102042223D1F04D
:1010300020910004203240F021E030E0FC013383B5
:10104000228380E090E015C080910104E82FF0E059
:10105000E956FC4F998190838F5F809301048093C0
:10106000000405C061E0CE0101960E948A0781E07C
:1010700090E00F90DF91CF910895089580E090E087
:101080000895CF93DF93EC01888581110FC081E033
:1010900088878A85882311F062E001C060E0898535
:1010A0000E94430F8FE090E00197F1F789850E943D
:1010B000EA0E2B8530E041E08217930709F440E007
:1010C000842FDF91CF9108951F920F920FB60F9248
:1010D00011246F927F928F929F92AF92BF92CF9284
:1010E000DF92EF92FF920F931F932F933F934F93B3
:1010F0005F936F937F938F939F93AF93BF93CF93A0
:10110000DF93EF93FF938091B9059091BA059C010D
:10111000215031093093BA052093B905892B09F084
:10112000B0C11092720078948091C100807F846079
:101130008093C10083E08093BF0088EE8093D1004C
:101140001092BF001092D20081E080930B01809139
:10115000BC059091BD05892B09F493C18091B70519
:1011600081118FC190900A018091B605882321F0EA
:101170008091B50581117BC17724739470ECA72E03
:101180007DE5B72EEAE06E2EF4E08F2EA0EDCA2E9C
:10119000A7E0DA2EB4E0EB2EF12C04EF11E0CFE063
:1011A000D0E00E941E062091BC053091BD052F5F46
:1011B0003F4F3093BD052093BC05853609F45EC0D2
:1011C0007CF5813609F49EC024F58C3309F452C0B5
:1011D0008E3309F44DC0813209F08FC080920A012C
:1011E000D0920701C0920601F0920901E092080135
:1011F0001093050100930401D0930301C0930201F1
:101200001092B60590900A01809104019091050119
:10121000C8CF833689F10CF478C000E022E077C0B3
:101220008D36A9F16CF4873679F15CF18C3609F0D2
:1012300064C00E943F0690930901809308014EC04C
:101240008237D1F14CF48F3609F057C00E943F0627
:10125000982E80930A01A5CF843789F1863709F04B
:101260004CC00E943F06909303018093020199CFE6
:10127000939497CF9A9495CF00E01FC000E024E0AC
:1012800046C000E025E043C000E027E040C00E94E7
:101290001E068C3619F41092B60504C07092B6057D
:1012A0001092B5058091BC059091BD050196909373
:1012B000BD058093BC0575CF01E020E028C00E94E9
:1012C0003F06BC01C5010E947425669EC001679E51
:1012D000900D1124909307018093060180910601DF
:1012E0009091070160910801709109010E94742595
:1012F000709305016093040154CF1092BD051092C4
:10130000BC05BFC000E029E002C000E02BE0122FC6
:101310003CE0939E100D11240E941E06982F977F8B
:10132000933259F48091BC059091BD05019690933C
:10133000BD058093BC051F5FEFCF8D3269F48091AE
:10134000BC059091BD0501969093BD058093BC05A9
:1013500011500E941E06F1CFC0910401D0910501E9
:101360008153883058F4C0910601D09107010E9442
:101370003F06BC01CE010E947425EB017E01F6946C
:10138000E7940E941E068E3261F48091BC05909114
:10139000BD0501969093BD058093BC05CE0DDF1D64
:1013A000EECFFE018091B605882349F0CE019695D7
:1013B00087958093B5058091B505E81BF109C0912B
:1013C0000201D0910301011104C01F3F11F0C111AE
:1013D00005C040E0BF0188EE93E046C0113130F017
:1013E00020EF210F203618F02FE501C020E0822FDA
:1013F0006CE00E946825682F74EF7603A001112429
:10140000BA01620F711D9B016C30710540F4220F0F
:10141000331FD901AE56BE4F2D913C9102C020E042
:1014200030E0873081F0082E02C0220F331F0A946B
:10143000E2F7823028F0C90105966AE070E00CC03E
:10144000C90190580CC0C90126E0880F991F2A9540
:10145000E1F7029665E070E00E947425CB014C2F05
:10146000C03108F04FE0BF010E9467060AC06091DA
:10147000B50570E040E088EE93E00E9467061092A8
:10148000B505FF91EF91DF91CF91BF91AF919F9102
:101490008F917F916F915F914F913F912F911F910C
:1014A0000F91FF90EF90DF90CF90BF90AF909F9003
:1014B0008F907F906F900F900FBE0F901F90189598
:1014C0001F920F920FB60F9211242F933F934F93B9
:1014D0005F936F937F938F939F93AF93BF93EF939C
:1014E000FF938091B900887F803609F49CC068F52D
:1014F000883209F45BC090F4803109F454C038F4A8
:10150000882309F4F6C0883009F44DC0F6C088314C
:1015100009F44CC0803209F45DC0EFC0803409F496
:1015200068C048F4803309F455C0883309F0E5C039
:101530008093DB03D8C0803509F44FC0883509F4A7
:101540005DC0883409F0D9C0D6C0883909F4C7C055
:10155000A8F4883709F467C038F4883609F463C002
:10156000803709F460C0C9C0883809F4B8C0803930
:1015700009F45FC0803809F0C0C05BC0803B09F44B
:1015800086C038F4803A09F466C0883A09F47FC00E
:10159000B4C0803C09F4A7C0883C09F4A4C0883BCF
:1015A00009F48AC0AAC08091D80310C09091DA03D0
:1015B0008091D903981770F5E091DA0381E08E0FDE
:1015C0008093DA03F0E0E954FC4F80818093BB0004
:1015D00085EC86C08093DB038EC0E091DA0381E066
:1015E0008E0F8093DA038091BB00F0E0E954FC4F4A
:1015F00080839091DA038091D9036EC0E091DA0381
:1016000081E08E0F8093DA038091BB00F0E0E95413
:10161000FC4F80838091DC0381116DC081E0809359
:10162000D70384EA61C083E08093DD031092B405A0
:10163000CFCF8091B405803208F051C0E091B4055D
:1016400081E08E0F8093B4058091BB00F0E0EC56F2
:10165000FA4F8083BDCF85EC8093BC001092DD03F0
:101660008091B405803230F4E091B405F0E0EC569E
:10167000FA4F10826091B40570E0E0919205F0910C
:10168000930584E995E009951092B40536C084E08D
:101690008093DD031092910510929005E0918E05E4
:1016A000F0918F05099580919005811105C081E029
:1016B0008093900510926E05E091910581E08E0F68
:1016C00080939105F0E0E259FA4F80818093BB004E
:1016D0009091910580919005981708F479CF85E84D
:1016E0008093BC000AC085EC8093BC001092DD039F
:1016F00004C01092DB030E948007FF91EF91BF911D
:10170000AF919F918F917F916F915F914F913F9199
:101710002F910F900FBE0F901F9018958091690523
:10172000811105C081E0809369050E943012F89410
:101730008091C0059091C105789490936B0580933A
:101740006A056EE873E00E9488257093AA02609390
:10175000A90280916905811105C081E08093690526
:101760000E943012F8948091BE059091BF05789444
:1017700090936D0580936C056EE873E00E94882558
:101780007093AC026093AB0208958F929F92AF92D8
:10179000BF92CF92DF92EF92FF920F931F930E941E
:1017A000B702E090B004F090B1048091A60290914D
:1017B000A702E81AF90AF0926805E09267050E940C
:1017C0008A0F2091A4023091A502AB01421B530B5A
:1017D0009A017093A5026093A402D7010E94A225EA
:1017E00020E030E040EE50E00E94A925EDE8AE2E6A
:1017F000F8E3BF2EACE0CA2EDD24D394E12CF12C0B
:1018000000E010E00E94E52549015A01809163053E
:1018100090916405A0916505B0916605880D991DAC
:10182000AA1DBB1D8093630590936405A093650575
:10183000B09366059D01552737FD5095452FA8E6C5
:10184000B1E00E94DD24BB2797FDB095AB2F8093BC
:10185000AD029093AE02A093AF02B093B0021F917D
:101860000F91FF90EF90DF90CF90BF90AF909F903F
:101870008F900895CF93DF9300D000D000D0CDB7E4
:10188000DEB761E0CE0101960E949201E1EBF2E049
:10189000AEE9B2E089819A812D913C911197821B2A
:1018A000930B918380838B819C8112962D913C9127
:1018B0001397821B930B938382838D819E81149651
:1018C0002D913C911597821B930B958384832696CB
:1018D0000FB6F894DEBF0FBECDBFDF91CF91089554
:1018E000882311F0479A01C047983F9A0895809144
:1018F000B1029091B2028D529140873C9105B0F4B3
:1019000082E58093A80281E00E94700C8AE492E054
:101910000E9470018091000190910101BC0197FF2C
:1019200002C06F5F7F4F759567951CC08091B502AF
:101930009091B6028D529140873C9105D8F48CE489
:101940008093A80281E00E94700C87E692E00E94DA
:1019500070016091000170910101CB0177FD01964A
:10196000959587950E949C1164E670E080E090E078
:101970000C94AF0F8091B3029091B4028D529140BC
:10198000873C910578F582E48093A8022898209AF4
:1019900083E892E00E94700187E092E00E9470016B
:1019A0008091B1029091B2028C329140B4F4809156
:1019B000B5029091B6028C3291407CF48091000186
:1019C0009091010197FD0196959587959195819547
:1019D0009109BC010E949C11E3CF64EF71E080E0AB
:1019E00090E0C6CF86E48093A8025D98559A82E97C
:1019F00092E00E9470018091000190910101BC0170
:101A00000C949C11CF92DF92EF92FF920F931F9351
:101A1000CF93DF936C017A018B01C0E0D0E0CE154B
:101A2000DF0589F0D8016D918D01D601ED91FC9112
:101A30000190F081E02DC6010995892B11F47E01FA
:101A400002C02196ECCFC701DF91CF911F910F917A
:101A5000FF90EF90DF90CF900895FC01538D448D5F
:101A6000252F30E0842F90E0821B930B541710F049
:101A7000CF96089501970895FC01918D828D981756
:101A800061F0828DDF01A80FB11D5D968C91928D62
:101A90009F5F9F73928F90E008958FEF9FEF08955F
:101AA000FC01918D828D981731F0828DE80FF11D28
:101AB000858D90E008958FEF9FEF0895FC01918D43
:101AC000228D892F90E0805C9F4F821B91098F733C
:101AD0009927089583E094E00E945E0D21E0892B10
:101AE00009F420E0822F0895FC01848DDF01A80F06
:101AF000B11DA35ABF4F2C91848D90E001968F7336
:101B00009927848FA689B7892C93A089B1898C9154
:101B100080648C93938D848D981306C00288F3891A
:101B2000E02D80818F7D80830895EF92FF920F9347
:101B30001F93CF93DF93EC0181E0888F9B8D8C8D79
:101B4000981305C0E889F989808185FD24C0F62EA7
:101B50000B8D10E00F5F1F4F0F731127E02E8C8D40
:101B6000E8120CC00FB607FCFACFE889F98980812A
:101B700085FFF5CFCE010E94740DF1CF8B8DFE0154
:101B8000E80FF11DE35AFF4FF0820B8FEA89FB89C2
:101B90008081806207C0EE89FF896083E889F989C6
:101BA00080818064808381E090E0DF91CF911F91FC
:101BB0000F91FF90EF900895CF93DF93EC01888D04
:101BC0008823C9F0EA89FB89808185FD05C0A88941
:101BD000B9898C9186FD0FC00FB607FCF5CF8081C7
:101BE00085FFF2CFA889B9898C9185FFEDCFCE0111
:101BF0000E94740DE7CFDF91CF91089580E090E0CF
:101C0000892B29F00E946A0D81110C94000008951F
:101C100090E0FC013197EF30F105B0F5EA5AFF4F43
:101C20000C949C25809180008F7703C08091800068
:101C30008F7D80938000089580918000877FF9CF09
:101C400084B58F7702C084B58F7D84BD089580915F
:101C500090008F7707C0809190008F7D03C08091A6
:101C60009000877F8093900008958091C0008F77C7
:101C700003C08091C0008F7D8093C0000895809143
:101C8000C200877F8093C200089508952E98269AF7
:101C90002D98259A2A98229A2998219A80EA809349
:101CA000800081E18093810080E991E0909387003A
:101CB00080938600109289001092880010928B0009
:101CC00010928A0008954FB141708CB186FB88272D
:101CD00080F984272091C4055091C3056091BE0509
:101CE0007091BF05982F9227292F30E0942F9527C8
:101CF000291B3109260F371F3093BF052093BE05DE
:101D00002091C3059091C405821729F0491719F055
:101D100091E09093C2058093C3054093C405089554
:101D20000E94A1281F920F920FB60F9211242F9399
:101D30003F934F935F936F937F938F939F93AF9353
:101D4000BF93EF93FF9383E094E00E94740DFF91A3
:101D5000EF91BF91AF919F918F917F916F915F9123
:101D60004F913F912F910F900FBE0F901F9018959C
:101D70001F920F920FB60F9211242F938F939F9360
:101D8000EF93FF93E0911304F09114048081E091AC
:101D90001904F0911A0482FD12C0908180911C04F4
:101DA0008F5F8F7320911D04821751F0E0911C0406
:101DB000F0E0ED5FFB4F958F80931C0401C08081A4
:101DC000FF91EF919F918F912F910F900FBE0F90E8
:101DD0001F901895CF93DF93282F30E0F901E25838
:101DE000FE4F8491F901E15AFE4FD491F901E05C74
:101DF000FE4FC491CC2391F081110E94080EEC2F6C
:101E0000F0E0EE0FFF1FEE5CFE4FA591B491EC9158
:101E1000ED2381E090E021F480E002C080E090E0DA
:101E2000DF91CF9108951F93CF93DF93282F30E058
:101E3000F901E258FE4F8491F901E15AFE4FD49125
:101E4000F901E05CFE4FC491CC23C9F0162F81113B
:101E50000E94080EEC2FF0E0EE0FFF1FEC5DFE4F2E
:101E6000A591B4918FB7F894111105C09C91ED2FF5
:101E7000E095E92302C0EC91ED2BEC938FBFDF914D
:101E8000CF911F910895CF93DF9390E0FC01E15A29
:101E9000FE4F2491FC01E05CFE4F8491882361F1A8
:101EA00090E0880F991FFC01EA5EFE4FC591D49126
:101EB000FC01EC5DFE4FA591B491611109C09FB783
:101EC000F8948881209582238883EC912E230BC07F
:101ED000623061F49FB7F8943881822F8095832314
:101EE0008883EC912E2B2C939FBF06C08FB7F8945C
:101EF000E8812E2B28838FBFDF91CF910895823008
:101F0000910538F0880F991F880F991F0597019741
:101F1000F1F708953FB7F8948091CE059091CF05E1
:101F2000A091D005B091D10526B5A89B05C02F3F43
:101F300019F00196A11DB11D3FBFBA2FA92F982FEF
:101F40008827820F911DA11DB11DBC01CD0142E06A
:101F5000660F771F881F991F4A95D1F708958F92B2
:101F60009F92AF92BF92CF92DF92EF92FF926B015E
:101F70007C010E948A0F4B015C01C114D104E10471
:101F8000F104F1F00E948A0FDC01CB018819990954
:101F9000AA09BB09883E9340A105B10570F321E071
:101FA000C21AD108E108F10888EE880E83E0981E75
:101FB000A11CB11CC114D104E104F10419F7DDCF57
:101FC000FF90EF90DF90CF90BF90AF909F908F9059
:101FD00008957F928F929F92AF92BF92CF92DF929D
:101FE000EF92FF920F931F93CF93DF93FC01228513
:101FF0003385232B09F479C07B01EC01D12C8C852E
:10200000D816F0F40D2D10E08E859F85F801EE0FA7
:10201000FF1FEE0DFF1D91838083EA85FB85E00F96
:10202000F11F61E080810E94130F8A859B85FC016E
:10203000E00FF11F61E080810E94430FD394DFCF56
:1020400083E290E00197F1F710E08C851817A8F46F
:10205000C12ED12CEA85FB85EC0DFD1D60E0808151
:102060000E94430F8A859B85FC01EC0DFD1D60E0FD
:1020700080810E94130F1F5FE8CF0E948A0F4B01DF
:102080005C010E948A0FAB01BC01481959096A0919
:102090007B098E859F85A0E0B0E0481759076A0745
:1020A0007B0718F50E948A0F6B01C818D908712C9C
:1020B0008C85781630F7072D10E0EA85FB85E00F58
:1020C000F11F80810E94EA0E892B51F4000F111F2D
:1020D000F701E00FF11F80819181C816D90610F039
:1020E0007394E6CFD182C082FBCFDF91CF911F9155
:1020F0000F91FF90EF90DF90CF90BF90AF909F90A7
:102100008F907F9008952FB7F8946091CA057091D1
:10211000CB058091CC059091CD052FBF08951F92DE
:102120000F920FB60F9211242F933F938F939F938B
:10213000AF93BF938091CA059091CB05A091CC0538
:10214000B091CD053091C90523E0230F2D3720F440
:102150000196A11DB11D05C026E8230F0296A11D01
:10216000B11D2093C9058093CA059093CB05A09318
:10217000CC05B093CD058091CE059091CF05A0916F
:10218000D005B091D1050196A11DB11D8093CE055A
:102190009093CF05A093D005B093D105BF91AF9197
:1021A0009F918F913F912F910F900FBE0F901F9095
:1021B00018951F920F920FB60F9211242F933F93F1
:1021C0004F935F936F937F938F939F93AF93BF933F
:1021D000EF93FF93E0911401F09115010995FF91A0
:1021E000EF91BF91AF919F918F917F916F915F918F
:1021F0004F913F912F910F900FBE0F901F90189508
:102200001F920F920FB60F9211242F933F934F936B
:102210005F936F937F938F939F93AF93BF93EF934E
:10222000FF93E0911201F09113010995FF91EF9155
:10223000BF91AF919F918F917F916F915F914F91DE
:102240003F912F910F900FBE0F901F9018951F92E6
:102250000F920FB60F9211242F933F934F935F93DA
:102260006F937F938F939F93AF93BF93EF93FF935E
:10227000E0911001F09111010995FF91EF91BF914B
:10228000AF919F918F917F916F915F914F913F910E
:102290002F910F900FBE0F901F9018951F920F92C5
:1022A0000FB60F9211242F933F934F935F936F9329
:1022B0007F938F939F93AF93BF93EF93FF93E0919F
:1022C0000E01F0910F010995FF91EF91BF91AF9130
:1022D0009F918F917F916F915F914F913F912F913E
:1022E0000F900FBE0F901F9018951F920F920FB670
:1022F0000F9211242F933F934F935F936F937F938C
:102300008F939F93AF93BF93EF93FF93E0910C0153
:10231000F0910D010995FF91EF91BF91AF919F91C0
:102320008F917F916F915F914F913F912F910F907E
:102330000FBE0F901F9018950F931F93CF93DF93AD
:102340008C01EB018091C805811105C081E080936B
:10235000C8050E94460E17FF05C011950195110989
:1023600081E001C080E0013991E0190714F000E933
:1023700011E010938B0000938A00882311F02A9AB1
:1023800001C02A98229A8091C805811105C081E078
:102390008093C8050E94460ED7FF05C0D195C19510
:1023A000D10981E001C080E0C13991E0D90714F082
:1023B000C0E9D1E0D0938900C0938800882311F050
:1023C000299A01C02998219ADF91CF911F910F91ED
:1023D000089546983E9AE0E9F0E082E0808310920A
:1023E0009100109271001082109299001092980042
:1023F00010929700109296001092950010929400FF
:1024000086988E980895FC01109271009B014617E2
:10241000570708F49A0146983E9890E890939000E8
:1024200010929100909392003E9AEF2B11F08E9AA9
:1024300001C08E98869A5093970040939600415021
:102440005109509395004093940030939900209344
:10245000980082E88093900089E18093910008952C
:1024600024982C9A6A98729A6E98769A8098889A8C
:1024700081E08093680090E190936B008BBB83E6D2
:102480009EE09093150180931401EAE6F0E08081CC
:102490008F7C80618083EE9A8CB182FB882780F9E3
:1024A0008093C70593B12091C70594FB882780F9D5
:1024B00082278093C6051092C1051092C005109224
:1024C000C5058FB181708093C4059CB12091C4056E
:1024D00096FB882780F982278093C3051092BF0559
:1024E0001092BE051092C20508951F920F920FB66A
:1024F0000F9211242F933F934F935F936F937F938A
:102500008F939F938CB190E095958795959587953E
:10251000482F417023B130E054E0359527955A9506
:10252000E1F78227932781702091C7055091C60556
:102530006091C0057091C105982F9227292F30E036
:10254000942F9527291B3109260F371F3093C1057A
:102550002093C0052091C6059091C705821729F0E8
:10256000491719F091E09093C5058093C6054093F3
:10257000C7059F918F917F916F915F914F913F918F
:102580002F910F900FBE0F901F901895FC01809116
:10259000DA05811103C08FEF9FEF08959FB7F8947C
:1025A00082E08093E9002091F20030E012161306D9
:1025B00014F421E030E02115310559F0289884E623
:1025C0008093D9058091F10080838091F200882367
:1025D00019F09FBFC90108958BE68093E800F9CFF9
:1025E0002FB7F89483E08093E9009091E800892F59
:1025F000807295FF04C09091F20080E4891B2FBF88
:1026000008958091E00581110DC082E08093DC0582
:1026100084E08093DD051092DF051092DE0581E0F5
:102620008093E0058CED95E00895CF93DF931F92A2
:10263000CDB7DEB76983DC01ED91FC910280F381B7
:10264000E02D41E050E0BE016F5F7F4F09950F9094
:10265000DF91CF91089583E08093E9008091F200AB
:10266000882319F08AE38093E80008950E94F0120D
:1026700090E00895CF93DF931F92CDB7DEB7FC01B2
:102680008485958597FD05C02FEF3FEF358724871B
:102690000BC0CE0101960E94C612019719F48981E0
:1026A00090E002C08FEF9FEF0F90DF91CF910895E0
:1026B0000F931F93CF93DF931F92CDB7DEB78C019B
:1026C000FC018485958597FF0EC0CE0101960E947E
:1026D000C612019719F4298130E002C02FEF3FEFB5
:1026E000F80135872487F801848595850F90DF915F
:1026F000CF911F910F910895FC018485958597FDD9
:102700000BC09FB7F89482E08093E9008091F200BB
:102710009FBF90E0019608959FB7F89482E0809360
:10272000E9008091F2009FBF90E008958F929F9200
:10273000AF92BF92CF92DF92EF92FF920F931F93CF
:10274000CF93DF935C016B017A0180912101882393
:1027500009F45BC08091DA05882309F456C08091A2
:10276000D80580FF05C08091E00082608093E00082
:10277000E70110E00AEF83E0882E9AE3992E209774
:10278000D9F10E94F01281110AC0015009F43DC034
:1027900061E070E080E090E00E94AF0FF0CF282F62
:1027A00030E0C217D3070CF48C2F4FB7F894809207
:1027B000E9009091E80095FF1DC0282F30E0C21B72
:1027C000D30BF601982F915020F081918093F10066
:1027D000FACFC20ED31E112319F09092E80009C05F
:1027E0008091E80085FD06C09092E80011E02097F6
:1027F00009F010E04FBFC3CF1111C3CF5D9884E63D
:102800008093DB051E141F0444F081E090E0F50185
:102810009383828380E090E001C0C701DF91CF9174
:102820001F910F91FF90EF90DF90CF90BF90AF90EE
:102830009F908F900895DF92EF92FF920F931F93D6
:10284000CF93DF93D82E8A017B01E40EF51EEB01B6
:10285000CE15DF0571F0D7FE03C0FE01849101C0E3
:1028600088810E94161721968111F2CF8FEF9FEF7A
:1028700001C0C801DF91CF911F910F91FF90EF90A0
:10288000DF9008950F931F93CF93DF931F92CDB7DF
:10289000DEB782E0898342E450E06DE971E080E8D0
:1028A0000E941B140E940113DC0112960D911C91D1
:1028B00013970115110569F0D801ED91FC91028083
:1028C000F381E02DBE016F5F7F4FC801099597FF2F
:1028D00007C089810F90DF91CF911F910F910895CB
:1028E000F80100851185E5CF1F920F920FB60F9268
:1028F00011248F939F938091E1009091E100937F49
:102900009093E10083FF0FC01092E90091E0909353
:10291000EB001092EC0092E39093ED001092DA0538
:1029200098E09093F00082FF20C093E09093E9003C
:102930009091F200992319F09AE39093E800909116
:10294000DB05992339F09091DB0591509093DB05DD
:10295000992389F19091D905992339F09091D9055E
:1029600091509093D905992341F184FF10C0809133
:10297000E2008E7E81608093E2008091E1008F7E94
:102980008093E1008091D8058E7E806111C080FF28
:1029900016C08091E2008E7E80618093E20080917B
:1029A000E1008E7E8093E1008091D8058E7E81606B
:1029B0008093D80504C05D9ACDCF289AD6CF9F9139
:1029C0008F910F900FBE0F901F9018951F920F922E
:1029D0000FB60F921124CF92DF92EF92FF920F93D6
:1029E0001F932F933F934F935F936F937F938F9397
:1029F0009F93AF93BF93EF93FF93CF93DF93CDB7A5
:102A0000DEB76C97DEBFCDBF1092E9008091E80081
:102A100083FFEDC168E0CE0145960E94441782EF26
:102A20008093E8008D8987FF05C09091E80090FFB2
:102A3000FCCF03C09EEF9093E800982F907609F0AA
:102A4000C6C09E892F89188D91110CC0803829F439
:102A50008091D7058093F10002C01092F10010928E
:102A6000F10048C1422F50E0512B913051F48111B7
:102A700041C14130510509F03DC18091D7058D7F9D
:102A80000BC0933061F4811135C14130510509F01B
:102A900031C18091D70582608093D7052BC19530D5
:102AA00041F48091E80080FFFCCF20682093E30090
:102AB00021C1963009F05FC0EB8CFC8C1092E900CC
:102AC0001092D5051092D405123091F51092D305CD
:102AD0001092D2050E94421499E0BE016F5F7F4FB1
:102AE000DB01E92F1D92EA95E9F799831A8391E0BA
:102AF0009E8390EA98879AEF99872091D405309128
:102B0000D505275F3F4F3C832B838D831092E900CF
:102B10001092D5051092D405F092D305E092D2051B
:102B200049E050E080E00E941B140E944214E2C081
:102B3000F092D305E092D2050E940113DC011296B7
:102B4000ED90FC901397E114F10409F4C0C0D70193
:102B5000ED91FC910480F581E02DBE016B5E7F4F0D
:102B6000C7010995009719F00CF0C4C0C7C0F70160
:102B7000E084F184E8CF973009F4C0C0983021F4A4
:102B800081E08093F100B6C0993009F0B3C0837042
:102B900009F0B4C0EBEAF1E081E021E036E3908196
:102BA000992361F08093E9002093EB009191909339
:102BB000EC003093ED008F5F873089F78EE78093CC
:102BC000EA001092EA008F898093DA0593C08B8D1A
:102BD0009C8D1092E9001092D5051092D405909327
:102BE000D3058093D205898D811156C08E899D8928
:102BF000913A59F4813209F081C047E050E06AE12E
:102C000071E080E00E941B1475C0913209F076C01B
:102C1000833289F4888D90E0982F88272F89822B22
:102C2000A0E0B0E08093160190931701A0931801E3
:102C3000B09319015FC0803269F48091E80082FF8F
:102C4000FCCF67E08AE191E00E9444178BEF80930C
:102C5000E80006C0823209F04DC08F8980932101BF
:102C60008091D605882319F0EEEFFAE002C0E0E08B
:102C7000F8E080911A0190911B01A0911C01B09184
:102C80001D01803B9440A105B10509F07BC08091F6
:102C9000210180FF93C076C00E940113DC011296CF
:102CA0000D911C9113970115110541F1D801ED917A
:102CB000FC910190F081E02DBE016B5E7F4FC80159
:102CC0000995811117C0F80100851185ECCF1130ED
:102CD00009F44EC0133091F48F89882309F445C05C
:102CE000823081F440E860E181E092E00E94772147
:102CF000882321F08EEF8093E80079C081E28093F1
:102D0000EB0075C0813029F440E86BE085EF91E07D
:102D1000EDCF833099F70E940113DC011296ED90FC
:102D2000FC9013978E010F5F1F4F6801E114F104AF
:102D300079F0D701ED91FC910680F781E02DB80183
:102D4000C7010995080F111DF701E084F184EECF4A
:102D5000D8011C92F60101900020E9F73197BF01DC
:102D60006C197D0940E0C601C1CF6FED71E002C072
:102D700063EE71E06115710509F2FB01449150E0C9
:102D800080E840CF0FB6F894A895809160008861E4
:102D900080936000109260000FBEA895EE3F2AE07D
:102DA000F20739F08091FE0A9091FF0A91838083A7
:102DB000A1CF1092FF0A1092FE0A9CCFEE3F8AE04C
:102DC000F80731F0808191819093FF0A8093FE0A89
:102DD00087E797E7918380839BE088E10FB6F894BB
:102DE000A895809360000FBE9093600083CF6C968F
:102DF0000FB6F894DEBF0FBECDBFDF91CF91FF912C
:102E0000EF91BF91AF919F918F917F916F915F9162
:102E10004F913F912F911F910F91FF90EF90DF9075
:102E2000CF900F900FBE0F901F9018954091D40532
:102E30005091D5052091D2053091D3054217530703
:102E4000B4F49091E8009570E1F39091E80092FD60
:102E500019C08093F1008091D4059091D505019619
:102E60008F739927892B19F48EEF8093E800809156
:102E7000D4059091D50501969093D5058093D405FE
:102E800081E0089580E00895615030F02091F100D4
:102E9000FC0120830196F8CF289884E68093D90519
:102EA0000895CF93DF93CDB7DEB7C257D1090FB6E0
:102EB000F894DEBF0FBECDBF789484B5826084BD28
:102EC00084B5816084BD85B5826085BD85B581602E
:102ED00085BD80916E00816080936E0010928100AC
:102EE0008091810082608093810080918100816067
:102EF0008093810080918000816080938000809128
:102F00009100826080939100809191008160809314
:102F10009100809190008160809390008091C10029
:102F200084608093C1008091C10082608093C10061
:102F30008091C10081608093C1008091C300816055
:102F40008093C3008091C00082608093C000809114
:102F5000C20081608093C20080917A008460809377
:102F60007A0080917A00826080937A0080917A0062
:102F7000816080937A0080917A00806880937A00E3
:102F80001092DA051092D7051092D8058091D700DB
:102F900081608093D70080EA8093D80089B58061F2
:102FA00089BD89B5826089BD09B400FEFDCF61E0AD
:102FB00070E080E090E00E94AF0F8091D8008F7C9D
:102FC00080618093D8008091E000807F8093E00052
:102FD0008091E1008E7E8093E1008DE08093E2009D
:102FE000559A209AEEEFFFE7859194918B3F9C4D87
:102FF00019F481E08093D605E0911304F091140454
:1030000082E08083E0910F04F09110041082E0913F
:103010001104F09112048FEC808310921B04E09154
:103020001704F091180486E08083E0911504F09174
:103030001604808180618083E0911504F09116046C
:10304000808188608083E0911504F091160480816E
:1030500080688083E0911504F091160480818F7D53
:10306000808383E094E00E945E0D892B21F081EB48
:1030700091E00E94700188EC91E00E947001109232
:10308000DF031092DE0310920104109200041092EC
:10309000DD0381E08093DC031092D70361E082E0DE
:1030A0000E94130F61E083E00E94130F8091B9002A
:1030B0008E7F8093B9008091B9008D7F8093B90095
:1030C00088E48093B80085E48093BC0064EF71E0ED
:1030D00080E090E00E94AF0F0E948A0F7093B802C8
:1030E0006093B7028BE08093080569E070E08091FF
:1030F0000505909106050E94D727FC01009769F00D
:10310000909306058093050583E08093070584E18D
:10311000808386E1838384E0868381E00E94700C53
:1031200082E1898385E18A838CE08B831092F604A7
:103130001092F5041092F8041092F7041092FA0419
:103140001092F9041092FC041092FB0410920405F2
:103150001092030583E08093FF048091FD04909119
:10316000FE04892B11F080E00BC083E090E00E9408
:10317000AA269093FE048093FD04892BA1F719C021
:103180009091FF04891790F4282F30E0E091FD041E
:10319000F091FE04E20FF31FA1E0B0E0AC0FBD1F01
:1031A000A20FB31F9C9190838F5FEACF8BE0809337
:1031B000000580ED97E0909302058093010531EEC4
:1031C000A2963FAFA297412C512C3201812C912C19
:1031D0005401C12CD12C7601809100019091010104
:1031E000A2964FADA2974C3328F466277727681B29
:1031F000790B04C0BC019195819591090E949C11A5
:1032000061E08EE992E00E94920180919E0290918D
:103210009F02C80ED91EE11CF11C8091A002909162
:10322000A102880E991EA11CB11C8091A20290914E
:10323000A302480E591E611C711C8091F7049091E5
:10324000F804892B39F08091F5049091F604892BCC
:10325000D1F41CC00091FF0410E0C801880F991F31
:103260000E94AA269093F8048093F704009709F42B
:10327000C5C0FC0180E090E08017910724F711920F
:1032800011920196F9CF00E010E01DC00091FF04FB
:1032900010E0C801880F991F0E94AA269093F60497
:1032A0008093F504009709F4A9C02091010530919D
:1032B0000205FC0180E090E08017910724F721933C
:1032C00031930196F9CF61E0CE018F5B9F4F0E9451
:1032D00092018091FF04A82FB0E0AD96BFAFAEAFD2
:1032E000AD97FE013196AB96FFAFEEAFAB97E05CCA
:1032F000FF4F9E012F5D3F4F1901A901CE0101969D
:10330000E3969FAF8EAFE39760E070E0AD968EAD31
:103310009FADAD9768177907BCF501151105A1F0B0
:10332000DA012D913C91808191812817390760F055
:10333000E396AEADBFADE3972D913C918081918135
:103340008217930748F010C080819181DA018D9334
:103350009C930115110561F780819181E396AEADD3
:10336000BFADE3978D939C936F5F7F4FE3962EAD38
:103370003FADE3972E5F3F4FE3963FAF2EAFE3970E
:1033800032964E5F5F4FC2CF0F5F1F4F0A3011055D
:1033900009F099CF6091F5047091F604A091F704BB
:1033A000B091F80480E090E02091FF0430E08217B3
:1033B000930724F5AB96EEADFFADAB97219131911C
:1033C000AB96FFAFEEAFAB974D915C911197421763
:1033D000530718F411963C932E93F10121913191EA
:1033E0001F01FB01408151812417350710F43183FF
:1033F000208301966E5F7F4F1296D6CFA2962FAD97
:10340000A2972F5FA2962FAFA297293509F0E4CE9D
:1034100080E00E94700C60E070E080E090E00E942C
:103420009C11C701B60128E730E040E050E00E945F
:10343000272530939F0220939E02C501B40128E7FF
:1034400030E040E050E00E9427253093A102209315
:10345000A002C301B20128E730E040E050E00E9442
:1034600027253093A3022093A20281E00E94700CD2
:103470008BE60E944B038F3F3FEF930719F021E04B
:1034800030E013C08AE60E944B038F3F3FEF930763
:1034900051F489E60E944B03833D910509F088C0F1
:1034A00021E030E08EC020E030E0873D910509F456
:1034B00073C081E090E09093B4048093B3040197CB
:1034C000029738F42130310511F08AE608C08BE606
:1034D00006C02130310511F088E601C089E68093ED
:1034E000B5046FEF80E20E942E0360E283E20E9447
:1034F0002E0360E084E20E942E0300E014E0C12C61
:10350000D12C76018091B5040E94050267E280EA21
:1035100094E00E940E080E945A028093B20461E077
:103520008091B5040E940F0280EA94E00E94C207D5
:103530000E945A020E94B7028091B0049091B10497
:10354000092E000CAA0BBB0BC80ED91EEA1EFB1ECF
:1035500001501109B9F6C701B60120E034E040E09E
:1035600050E00E94BE243093A7022093A6020E943E
:103570008A0F7093A5026093A40280E00E94700CF1
:1035800081E00E94700C6FE070E08DE10E94EE041B
:103590008934910521F4D3C582E090E08CCF6FE0AF
:1035A00070E08EE10E94EE048934910569F4CAC589
:1035B00088E60E944B03833D910509F092CF20E0FD
:1035C00030E080E090E077CF60E270E089E10E9437
:1035D000EE04019661F06FE070E08EE10E94EE046F
:1035E00021E030E0CC97D1F080E090E019C060E2BB
:1035F00070E088E10E94EE04019609F44AC06FE091
:1036000070E08EE10E94EE0431E020E0CC9709F0FA
:1036100030E0832F922F20E030E002C082E090E083
:103620009093D3048093D2048230910509F41EC490
:103630008330910509F041C42130310509F46DC48E
:103640008EE18093D5048093D40488E090E0909339
:10365000DB048093DA0489E090E09093D9048093AE
:10366000D8048AE090E09093DF048093DE048BE03E
:1036700090E09093DD048093DC048CE090E09093E4
:10368000E3048093E2048DE090E09093E104809362
:10369000E0048091D2049091D30483309105D1F459
:1036A00060E081E20E94E10467E580E20E94E104BB
:1036B00064E684E20E94E10460E285E20E94E104A3
:1036C00060E086E20E94E10400E014E060E070E067
:1036D000CB011DC0029731F468E083E20E94C4046C
:1036E00067E405C060E083E20E94C40467E280E210
:1036F0000E94C4046CE080E00E94A70460E281E0C4
:103700000E94A70460E082E00E94A704DDCFAE968D
:103710006FAFAE97AF967FAFAF97E0968FAFE09762
:10372000E1969FAFE1970E942E040E946B03C09028
:10373000B904D090BA040D2C000CEE08FF08AE9628
:103740006FADAE97AF967FADAF97E0968FADE09738
:10375000E1969FADE1976C0D7D1D8E1D9F1D015063
:103760001109A9F620E034E040E050E00E94BE24B8
:103770003093C4022093C3020E948A0F7093C20246
:103780006093C10280E00E94700C8BED91E00E947A
:1037900070015D98559AE091E704F091E80401907A
:1037A000F081E02D87EE94E009958823A1F36AE08B
:1037B00070E080E090E00E94AF0FE091E704F091AC
:1037C000E8040190F081E02D87EE94E009958823CC
:1037D00011F3E091E704F091E8040190F081E02D0D
:1037E00087EE94E009958111F4CF6AE070E080E003
:1037F00090E00E94AF0FE091E704F091E80401909F
:10380000F081E02D87EE94E009958111E2CF0E94CE
:103810008310611571058105910511F00E94072241
:1038200064EF71E080E090E00E94AF0F72E0872EBD
:10383000912CA12CB12CE3E04E2E512C612C712C3B
:10384000F4E62F2E312CA8ECCA2E5D9A559A80E012
:103850000E94700C289A209A0E948A0F2091B70229
:103860003091B802DB01A21BB30BB0938E03A0937F
:103870008D037093B8026093B7020E943A0C0E94C5
:103880001A0584E10E94460110910705811758F43A
:10389000E0910505F0910605B3E08B9FE00DF11D69
:1038A0001124818101C080E080938F0386E10E9412
:1038B0004601811758F4E0910505F091060523E0D3
:1038C000829FE00DF11D1124D18001C0D12CD09236
:1038D000900386E10E944601811758F4E0910505A6
:1038E000F091060533E0839FE00DF11D1124128154
:1038F00001C010E0109391030E945C018093920339
:103900000E94C50B0E942E040E946B03E090B90434
:10391000F090BA048091C3029091C402E81AF90AA7
:10392000F0929403E09293030E948A0F2091C102C7
:103930003091C202AB01421B530B7093C2026093E1
:10394000C1029A01D7010E94A2259A0140E050E0ED
:103950000E94A9250EE00E948326A2962FAFA2976F
:10396000A3963FAFA397A4964FAFA497A5965FAF3A
:10397000A597A6966FAFA697A7967FAFA797A8968D
:103980008FAFA897A9969FAFA9978091BD029091FC
:10399000BE02A091BF02B091C002A5962CAD3DAD74
:1039A0004EAD5FADA597280F391F4A1F5B1F2093AF
:1039B000BD023093BE024093BF025093C002A8EEF6
:1039C000B3E00E94DD2429E030E040E050E00E94B6
:1039D000BE242093B9023093BA024093BB025093A5
:1039E000BC020E948E0B83E094E00E943C0D9093F9
:1039F000960380939503019731F53092010120924F
:103A0000000149EEE41643E0F4063CF060E070E0AB
:103A100080E090E00E949C11D1C154E05D15B0F3AC
:103A20001530A0F78091B1029091B202893E934087
:103A30006CF78091B5029091B602893E934034F7BD
:103A40000E94770CBBC1E9EEEE16E3E0FE060CF433
:103A50003DC0F8E5F093A80285EF91E00E94700167
:103A600087E092E00E9470012898209A60E070E060
:103A700080E090E00E949C1164EF71E080E090E0B3
:103A80000E94AF0F8091B1029091B2028C329140AE
:103A9000B4F48091B5029091B6028C3291407CF4DE
:103AA000809100019091010197FD01969595879570
:103AB000919581959109BC010E949C11E3CF64EF1F
:103AC00071E080E090E00E94AF0F78C146E0D4162C
:103AD00009F49CCF163009F499CF55E0D51619F0AA
:103AE000153009F01DC185E58093A80289E092E0B8
:103AF0000E94700187E092E00E94700181E00E94C4
:103B0000700C1092AD021092AE021092AF021092A1
:103B1000B0020E94C50B8091AD029091AE02A091BF
:103B2000AF02B091B0028D97A105B10574F40E9467
:103B3000C50B6091000170910101CB0177FD0196E9
:103B4000959587950E949C11E6CF0E943A0C809132
:103B5000B5029091B6028C32914054F40E943A0C16
:103B60008091000190910101BC010E949C11EFCF56
:103B70000E94C50B8091AD029091AE02A091AF0260
:103B8000B091B002181619061A061B0684F40E949A
:103B9000C50B8091000190910101BC0197FF02C00B
:103BA0006F5F7F4F759567950E949C11E3CF0091E1
:103BB000000110910101B801C8010E949C110E94EE
:103BC0001A0586E10E944601E09007058E1558F41B
:103BD000E0910505F0910605B3E08B9FE00DF11D26
:103BE0001124F18001C0F12CF092900386E10E9433
:103BF00046018E1558F4E0910505F091060523E085
:103C0000829FE00DF11D1124828101C080E080932C
:103C1000910333E03F1568F4843058F01092AD0200
:103C20001092AE021092AF021092B0020E94C50B29
:103C300033C0B801C8010E949C1168EE73E080E0B7
:103C400090E00E94AF0F0E941A050E945C018093D1
:103C5000920380919203853008F380910001909146
:103C60000101BC010E949C110E941A050E945C0186
:103C7000809392030E94770CECCF0E94C50B809139
:103C8000000190910101BC0197FF02C06F5F7F4F5F
:103C9000759567950E949C118091AD029091AE023E
:103CA000A091AF02B091B002843D9F4FAF4FBF4F84
:103CB00024F70E943A0C8091B1029091B2028C32AA
:103CC000914054F40E943A0C8091000190910101BE
:103CD000BC010E949C11EFCF0E94C50B8091AD02E8
:103CE0009091AE02A091AF02B091B002B7FF0EC0AA
:103CF0000E94C50B6091000170910101CB0177FD1D
:103D00000196959587950E949C11E8CF80910001BE
:103D100090910101BC010E949C118CE192E04CC089
:103D20008091B1029091B202893E934044F4809117
:103D3000B5029091B602893E93400CF481CEE1E445
:103D4000E093A80281E00E94700C8DE292E00E9454
:103D5000700187E092E00E94700181E02091B10241
:103D60003091B202293E33400CF480E02091B5023C
:103D70003091B602293E33400CF0D9C0882349F077
:103D80000E940222A50194010E94BE24613009F420
:103D9000E4C0809100019091010197FD01969595F5
:103DA0008795BC010E949C1164EF71E080E090E077
:103DB0000E94AF0F86E392E00E94700180918E0313
:103DC0008F9380918D038F938091B0028F93809118
:103DD000AF028F938091AE028F938091AD028F934B
:103DE0008091AC028F938091AB028F938091AA0255
:103DF0008F938091A9028F938091B6028F938091C7
:103E0000B5028F938091B4028F938091B3028F9308
:103E10008091B2028F938091B1028F93809192032F
:103E20001F928F93809191031F928F9380919003A3
:103E30001F928F9380918F031F928F93AAECB0E013
:103E4000BF93AF931F92CF92A5ECB2E0BF93AF9315
:103E50000E94102285EC92E00E9470010FB6F89447
:103E6000DEBF0FBECDBF0E94FE0DEFCC89E1809377
:103E7000D4048EE18093D50483E090E09093D9043C
:103E80008093D80484E090E09093DB048093DA047C
:103E900087E090E09093DD048093DC0488E090E07C
:103EA0009093DF048093DE0485E090E09093E1043A
:103EB0008093E00486E090E02BC0019781F12130EF
:103EC000310599F188E18093D4048EE18093D50483
:103ED00083E090E09093D9048093D80484E090E04C
:103EE0009093DB048093DA0485E090E09093DD0406
:103EF0008093DC0486E090E09093DF048093DE04FE
:103F000087E090E09093E1048093E00488E090E003
:103F10009093E3048093E204BCCB8DE192CB2130FB
:103F2000310509F4A3CF88E1A2CF89E1CCCF882362
:103F300059F00E940222A50194010E94BE246F5FE5
:103F4000613009F09BC009C00E940222A3019201C6
:103F50000E94BE246130C1F391C01092AA02109257
:103F6000A9021092AC021092AB028091A90290912A
:103F7000AA02019711F18091AB029091AC020197D6
:103F8000E1F08091B1029091B2028C329140ACF498
:103F90008091B5029091B6028C32914074F40E94E7
:103FA0008E0B809100019091010197FD01969595EE
:103FB0008795BC010E949C11D8CF1092AD0210923F
:103FC000AE021092AF021092B0020E94C50B809117
:103FD000AD029091AE02A091AF02B091B0028A35CD
:103FE0009105A105B10509F4D4CE0E94C50B20911D
:103FF000B1023091B2022D52314080910001909176
:104000000101273C310528F497FD01969595879588
:1040100012C02091B3023091B4022D523140273C9E
:10402000310558F497FD0396959587959595879555
:10403000919581959109BC011EC02091B5023091E6
:10404000B6022D523140273C310540F497FD0196D0
:10405000BC017595679580E090E00DC0BC0197FFAD
:1040600002C06F5F7F4F7595679597FD0396959595
:104070008795959587950E949C11A9CF623009F08C
:1040800088CE1092AD021092AE021092AF02109242
:10409000B0020E94C50B8091AD029091AE02A0913A
:1040A000AF02B091B002863A9F4FAF4FBF4F09F4B5
:1040B00070CE0E94C50B2091B1023091B2022D52F8
:1040C00031408091000190910101273C310528F495
:1040D00097FD019660E070E02DC02091B302309111
:1040E000B4022D523140273C310550F497FD039620
:1040F00095958795959587959195819591090DC091
:104100002091B5023091B6022D523140273C310545
:1041100030F497FD019695958795BC010DC0BC01C3
:1041200097FF02C06D5F7F4F759567957595679591
:1041300097FD0196959587950E949C11ACCF21E043
:1041400030E002C020E030E083E090E069CAE3E1C3
:10415000F5E01382128288EE93E0A0E0B0E0848361
:104160009583A683B78328E431E0318320832FEF42
:104170003FEF35872487E3E0F4E0138212828483E3
:104180009583A683B7832AE531E0318320832DEC24
:1041900030E0358724872CEC30E03787268728EC01
:1041A00030E0318B208B29EC30E0338B228B2AECF2
:1041B00030E0358B248B2EEC30E0378B268B118E44
:1041C000128E138E148EE0EAF4E01382128284833E
:1041D0009583A683B7838CE691E091838083E5E0A5
:1041E000F5E01182108212828FEF83831582148290
:1041F000168285EA91E09287818782E492E0948733
:10420000838784EA91E090878783E3EFF4E0138269
:1042100012821582148217821682118610861386E6
:10422000128680E991E091838083E7EEF4E01282C8
:10423000158210868EE0818781E0828783878EE7F2
:1042400091E09183808386E0ECE2F1E0ABECB4E0B6
:1042500001900D928A95E1F786E0E2E3F1E0A5ECAA
:10426000B4E001900D928A95E1F7E9EBF4E084E087
:1042700090E0928F818F14A613A615A6ECEAF4E0C5
:1042800083E090E0908787831386128614860895D2
:104290008AE891E09093F4048093F3048091FD0404
:1042A0009091FE04009711F00E943F278091F7043F
:1042B0009091F804009711F00E943F278091FB0431
:1042C0009091FC04009711F00E943F278091F50423
:1042D0009091F604009711F00E943F278091F90415
:1042E0009091FA04009711F00C943F270895CF9213
:1042F000DF92EF92FF920F931F93CF93DF931F9262
:10430000CDB7DEB7182F062FE42E862F880F8E5FCD
:1043100099830E94161783E00E941617F12EC12E72
:104320009981D92E8C2D8F19801798F4F601E7FE0C
:1043300002C0849101C080810E941617182F80E06E
:104340000E9416178123FFEFCF1ADF0A8111EACFEF
:1043500001C081E00F90DF91CF911F910F91FF90ED
:10436000EF90DF90CF9008958F929F92AF92BF927F
:10437000CF92DF92EF92FF92CF93DF93EC016881AF
:1043800079818A819B81611571058105910521F4EF
:1043900064E279ED8BE597E02DE133EF41E050E009
:1043A0000E94BE2449015A019B01AC01A7EAB1E475
:1043B0000E94DD246B017C01ACEEB4EFA5019401F9
:1043C0000E94EB24DC01CB018C0D9D1DAE1DBF1D99
:1043D000B7FF03C00197A109B04888839983AA83D6
:1043E000BB83BC01CD019F77DF91CF91FF90EF9010
:1043F000DF90CF90BF90AF909F908F9008950E94D4
:10440000B421089582E291E00E94B421089560935E
:104410002201709323018093240190932501089534
:10442000AEE0B0E0E6E1F2E20C94FE240D891E89D4
:104430008F89988D2EE02C831A83098397FF02C001
:1044400080E090E801979E838D83AE01455E5F4FCB
:10445000698D7A8DCE0101960E9440224D815E8148
:1044600057FD0AC02F813885421753070CF49A0173
:10447000F801E20FF31F10822E96E4E00C941A2547
:10448000ACE0B0E0E6E4F2E20C94F0247C016B01D5
:104490008A01FC0117821682838181FFBDC1CE0192
:1044A00001964C01F7019381F60193FD859193FFED
:1044B00081916F01882309F4ABC1853239F493FDF2
:1044C000859193FF81916F01853229F4B70190E0C6
:1044D0000E942824E7CF512C312C20E02032A0F478
:1044E0008B3269F030F4803259F0833269F4206104
:1044F0002CC08D3239F0803339F4216026C022601F
:10450000246023C0286021C027FD27C030ED380F6C
:104510003A3078F426FF06C0FAE05F9E300D112491
:10452000532E13C08AE0389E300D1124332E2062A2
:104530000CC08E3221F426FD6BC1206406C08C367F
:1045400011F4206802C0883641F4F60193FD85918C
:1045500093FF81916F018111C1CF982F9F7D955459
:10456000933028F40C5F1F4FFFE3F9830DC08336AF
:1045700031F0833771F0833509F05BC022C0F80158
:10458000808189830E5F1F4F44244394512C540132
:1045900015C03801F2E06F0E711CF801A080B180E7
:1045A00026FF03C0652D70E002C06FEF7FEFC501ED
:1045B0002C870E941D242C0183012C852F77222E0D
:1045C00017C03801F2E06F0E711CF801A080B180B5
:1045D00026FF03C0652D70E002C06FEF7FEFC501BD
:1045E0002C870E9412242C012C852068222E830106
:1045F00023FC1BC0832D90E048165906B0F4B70188
:1046000080E290E00E9428243A94F4CFF50127FC40
:10461000859127FE81915F01B70190E00E942824D7
:1046200031103A94F1E04F1A51084114510471F7D6
:10463000E5C0843611F0893639F5F80127FF07C047
:1046400060817181828193810C5F1F4F08C06081FE
:104650007181072E000C880B990B0E5F1F4F2F7670
:10466000722E97FF09C090958095709561957F4F48
:104670008F4F9F4F2068722E2AE030E0A4010E94E5
:104680006024A82EA81844C0853729F42F7EB22EA6
:104690002AE030E025C0F22FF97FBF2E8F36C1F01F
:1046A00018F4883579F0B4C0803719F0883721F0D4
:1046B000AFC02F2F2061B22EB4FE0DC08B2D8460B1
:1046C000B82E09C024FF0AC09F2F9660B92E06C0DD
:1046D00028E030E005C020E130E002C020E132E017
:1046E000F801B7FE07C060817181828193810C5F00
:1046F0001F4F06C06081718180E090E00E5F1F4F08
:10470000A4010E946024A82EA818FB2DFF777F2EFD
:1047100076FE0BC0372D3E7FA51450F474FE0AC000
:1047200072FC08C0372D3E7E05C0BA2C372D03C061
:10473000BA2C01C0B52C34FF0DC0FE01EA0DF11DED
:104740008081803311F4397E09C032FF06C0B394F2
:10475000B39404C0832F867809F0B39433FD13C05B
:1047600030FF06C05A2CB31418F4530C5B18B32C4A
:10477000B31468F4B70180E290E03C870E942824DB
:10478000B3943C85F5CFB31410F43B1801C0312C21
:1047900034FF12C0B70180E390E03C870E942824D8
:1047A0003C8532FF17C031FD03C088E790E002C0AE
:1047B00088E590E0B7010CC0832F867859F031FF6F
:1047C00002C08BE201C080E237FD8DE2B70190E0CC
:1047D0000E942824A51438F4B70180E390E00E94D9
:1047E00028245A94F7CFAA94F401EA0DF11D808190
:1047F000B70190E00E942824A110F5CF332009F4DE
:1048000051CEB70180E290E00E9428243A94F6CF7E
:10481000F7018681978102C08FEF9FEF2C96E2E12E
:104820000C940C25FC010590615070400110D8F7E4
:10483000809590958E0F9F1F0895FC0161507040E8
:1048400001900110D8F7809590958E0F9F1F0895C5
:104850000F931F93CF93DF93FB01238121FD03C0AF
:104860008FEF9FEF28C022FF16C046815781248119
:1048700035814217530744F4A081B1819D012F5F18
:104880003F4F318320838C93268137812F5F3F4FA9
:104890003783268310C0EB01092F182F0084F18580
:1048A000E02D0995892BE1F68E819F8101969F83EA
:1048B0008E83812F902FDF91CF911F910F910895BB
:1048C000FA01AA27283051F1203181F1E8946F9341
:1048D0006E7F6E5F7F4F8F4F9F4FAF4FB1E03ED0E7
:1048E000B4E03CD0670F781F891F9A1FA11D680F85
:1048F000791F8A1F911DA11D6A0F711D811D911DB8
:10490000A11D20D009F468943F912AE0269F11242C
:104910003019305D3193DEF6CF010895462F477090
:10492000405D4193B3E00FD0C9F7F6CF462F4F70EB
:10493000405D4A3318F0495D31FD4052419302D049
:10494000A9F7EACFB4E0A6959795879577956795EF
:10495000BA95C9F700976105710508959B01AC01EF
:104960000A2E06945795479537952795BA95C9F716
:10497000620F731F841F951FA01D0895052E97FBBE
:104980001EF400940E94D52457FD07D00E942725CD
:1049900007FC03D04EF40C94D524509540953095E7
:1049A00021953F4F4F4F5F4F08959095809570959B
:1049B00061957F4F8F4F9F4F08950E944925A59F76
:1049C000900DB49F900DA49F800D911D112408950A
:1049D000B7FF0C94DD240E94DD24821B930B089505
:1049E0002F923F924F925F926F927F928F929F92FF
:1049F000AF92BF92CF92DF92EF92FF920F931F93ED
:104A0000CF93DF93CDB7DEB7CA1BDB0B0FB6F8949D
:104A1000DEBF0FBECDBF09942A88398848885F84DD
:104A20006E847D848C849B84AA84B984C884DF804E
:104A3000EE80FD800C811B81AA81B981CE0FD11D32
:104A40000FB6F894DEBF0FBECDBFED010895A1E211
:104A50001A2EAA1BBB1BFD010DC0AA1FBB1FEE1FF8
:104A6000FF1FA217B307E407F50720F0A21BB30B43
:104A7000E40BF50B661F771F881F991F1A9469F7BF
:104A800060957095809590959B01AC01BD01CF011B
:104A90000895A29FB001B39FC001A39F700D811D17
:104AA0001124911DB29F700D811D1124911D089537
:104AB000DB018F939F930E94DD24BF91AF91A29F52
:104AC000800D911DA39F900DB29F900D112408950C
:104AD000991B79E004C0991F961708F0961B881F50
:104AE0007A95C9F780950895AA1BBB1B51E107C0B1
:104AF000AA1FBB1FA617B70710F0A61BB70B881F6E
:104B0000991F5A95A9F780959095BC01CD010895FC
:104B100097FB072E16F4009407D077FD09D00E946A
:104B2000742507FC05D03EF4909581959F4F08951C
:104B3000709561957F4F0895EE0FFF1F0590F491DA
:104B4000E02D09940E944925B7FF0895821B930B1D
:104B5000089597FB57FF0C94B9259F938F930E945C
:104B6000B9256E1B7F0BAF91BF918A0B9B0B0895EC
:104B7000E894DF93CF93FC01DB010E9449257F93EA
:104B80006F93E9019A01AC01BF93AF933F932F93C9
:104B9000DF010E94492526F46C1B7D0B820B930BD1
:104BA0009E01EB01FC010E94A126AF91BF912F91C4
:104BB0003F910E94A126BE01CF01F9012F913F91A3
:104BC000CF91DF910895689401C0E894F92FF12BFB
:104BD00012F00C941726A0E0B0E0E1EFF5E20C949F
:104BE000F624092E059422F40E947326112392F4D0
:104BF000F0E80F26FFEFE094F09400951095B09444
:104C0000C094D094A194BF0ACF0ADF0AEF0AFF0A2A
:104C10000F0B1F0B0E94222607FC0E947326CDB7A4
:104C2000DEB7ECE00C941225689401C0E8948F92F2
:104C30009F92CF93DF930E942226DF91CF919F9086
:104C40008F90089588249924F401E401B0E49F939F
:104C5000AA279A158B049C04ED05FE05CF05D00705
:104C6000A10798F4AD2FDC2FCF2FFE2FE92D982C24
:104C7000892E982F872F762F652F542F432F322F71
:104C80002227B85031F7BF9127C01B2EBF91BB27F9
:104C9000220F331F441F551F661F771F881F991F40
:104CA000881C991CEE1FFF1FCC1FDD1FAA1FBB1FF6
:104CB0008A149B04EC05FD05CE05DF05A007B107AE
:104CC00048F08A189B08EC09FD09CE09DF09A00B02
:104CD000B10B21601A94E1F62EF49401AF01BE01EC
:104CE000CD01000C08956095709580959095309554
:104CF0004095509521953F4F4F4F5F4F6F4F7F4FDE
:104D00008F4F9F4F089597FB10F8169400080F934C
:104D1000083098F00850232F342F452F562F672F37
:104D2000782F892F902DF4CF0594979587957795B7
:104D3000679557954795379527950A95AAF70F9147
:104D400008950E944925460F571FC81FD91F08F410
:104D500031960895CF93DF938230910510F482E06D
:104D600090E0E091EA05F091EB0520E030E0C0E052
:104D7000D0E0309711F14081518148175907C0F0B8
:104D80004817590761F482819381209719F09B831A
:104D90008A832BC09093EB058093EA0526C02115EA
:104DA000310519F04217530718F49A01BE01DF01CB
:104DB000EF010280F381E02DDCCF2115310509F1EF
:104DC000281B390B2430310590F412968D919C915B
:104DD00013976115710521F0FB019383828304C051
:104DE0009093EB058093EA05FD01329644C0FD01E6
:104DF000E20FF31F81939193225031092D933C933D
:104E00003AC02091E8053091E905232B41F4209127
:104E10002801309129013093E9052093E80520917C
:104E20002601309127012115310541F42DB73EB7F8
:104E300040912A0150912B01241B350BE091E8058C
:104E4000F091E905E217F307A0F42E1B3F0B28179A
:104E5000390778F0AC014E5F5F4F2417350748F0F3
:104E60004E0F5F1F5093E9054093E805819391939E
:104E700002C0E0E0F0E0CF01DF91CF9108950F9301
:104E80001F93CF93DF93009709F48CC0FC013297F6
:104E9000138212820091EA051091EB0501151105AC
:104EA00081F420813181820F931F2091E805309198
:104EB000E9052817390779F5F093E905E093E80546
:104EC00071C0D80140E050E0AE17BF0750F4129611
:104ED0002D913C911397AD012115310509F1D901AF
:104EE000F3CF9D01DA013383228360817181860FC4
:104EF000971F8217930769F4EC0128813981260FE7
:104F0000371F2E5F3F4F318320838A819B8193839C
:104F10008283452B29F4F093EB05E093EA0542C028
:104F20001396FC93EE931297ED01499159919E01CE
:104F3000240F351FE217F30771F480819181840FEC
:104F4000951F029611969C938E938281938113965E
:104F50009C938E931297E0E0F0E0D80112968D9129
:104F60009C911397009719F0F8018C01F6CF8D9161
:104F70009C9198012E5F3F4F820F931F2091E8056F
:104F80003091E9052817390769F4309729F4109210
:104F9000EB051092EA0502C0138212821093E90514
:104FA0000093E805DF91CF911F910F910895A0E044
:104FB000B0E0EDEDF7E20C94F424EC01009721F45D
:104FC000CB010E94AA26B8C0FC01E60FF71F9C0186
:104FD00022503109E217F30708F4ACC0D9010D9152
:104FE0001C91119706171707B0F00530110508F44A
:104FF0009FC0C80104978617970708F499C002500C
:105000001109061B170B019311936D937C93CF012C
:105010000E943F278DC05B01A01AB10A4C01800E8F
:10502000911EA091EA05B091EB0540E050E0E12C23
:10503000F12C109709F44AC0A815B905D1F56D9067
:105040007C901197630182E0C80ED11CCA14DB0466
:1050500080F1A3014A195B096A0182E0C80ED11CE4
:105060001296BC9012971396AC91B5E0CB16D10472
:1050700040F0B282A38351834083D9016D937C9326
:105080000AC00E5F1F4FC301800F911FF90191836A
:105090008083EB2DFA2FE114F10431F0D701139640
:1050A000FC93EE93129744C0F093EB05E093EA056E
:1050B0003FC08D919C9111974817590708F4AC0196
:1050C0007D0112960D90BC91A02DB3CF8091E80583
:1050D0009091E90588159905E1F446175707C8F43A
:1050E0008091260190912701009741F48DB79EB7DA
:1050F00040912A0150912B01841B950BE817F90769
:10510000C8F4F093E905E093E805F9017183608341
:105110000FC0CB010E94AA267C01009759F0A8017C
:10512000BE010E94A628CE010E943F27C70104C0ED
:10513000CE0102C080E090E0CDB7DEB7EEE00C9487
:10514000102581E090E0F8940C94AF28FB01DC017D
:1051500002C001900D9241505040D8F7089511E0DF
:10516000CAE0D1E004C0FE010E949C252196CB300C
:08517000D107C9F7F894FFCF45
:10517800C8000F00F401D00704000401450E450ED5
:10518800450E450E450EFFFFFFFF00E10000000041
:105198000000010000000000EC0580000180018093
:1051A8000180FF7FFF7FFF7F04000F002000370092
:1051B80055007800000000001513961336132B13C2
:1051C8007C133A13581300000000950D020D2D0DA5
:1051D800DC0D5E0D3C0D500D000000000E08DE07D2
:1051E8003E08B207D607C207B3070000000041080F
:1051F80000000000E90F00000000900E0000000011
:10520800E90F9C01B501CF01EA0107022602470216
:1052180069028E02B502DE020A0300C18081000025
:105228000056657262696E64756E6720686572679C
:10523800657374656C6C740053656E736F726B6123
:105248006C696272696572756E67005A756D6F2058
:105258006265726569742C20737461727465206D5F
:1052680069742041004B6F6C6C6973696F6E2065BF
:10527800726B616E6E7400310048696E6465726E9F
:10528800697320756D66616872656E00556D66613B
:105298006872656E206265656E646574004162625D
:1052A800696567656E00416262696567656E20625F
:1052B80065656E646574000D0A0053707572206E22
:1052C80061636820726563687473206B6F727269BA
:1052D80067696572656E0053707572206E616368E8
:1052E800206C696E6B73206B6F7272696769657287
:1052F800656E0053707572207665726C61737365A4
:0E5308006E005370757220666F6C67656E00E4
:00000001FF
